:020000040800F2
:10000000101B0020CD000008FD0F0008ED0F0008B8
:1000100000000000000000000000000000000000E0
:10002000000000000000000000000000FF0F0008BA
:10003000000000000000000011330008D142000859
:10004000DF00000800000000DF000008DF000008FB
:10005000DF000008DF000008DF000008DF00000804
:1000600000000000DF000008B9040008590500087E
:10007000DF000008DF000008DF00000800000000CB
:10008000DF000008E143000800000000DF00000876
:10009000DF000008DF000008DF000008DF000008C4
:1000A000DF0000089D3C0008DF000008F94300085D
:1000B000814400080348854600F0D6F80048004710
:1000C000BD4D0008101B00200844F047044880473D
:1000D00004480047FEE7FEE7FEE7FEE7FEE7FEE72F
:1000E00085430008B500000830B50B4601460020E6
:1000F0002022012409E00D46D5409D4205D31D462E
:100100009540491B2546954040191546521E002D25
:10011000F1DC30BD70B500242546002801DA012449
:100120004042002901DA01254942FFF7DDFFAC42D8
:1001300000D04042002C00D0494270BDF8B50024E8
:100140002546002904DA0E46012400214042B1412F
:10015000002B04DA1E46002352420125B34100F071
:1001600052F88C4617461E46AC4203D0002540424A
:100170008D41AC46002C02D0002657429E4161467C
:100180003A46334601B0F0BD10B5202A04DB0846DC
:10019000203AD040002110BD0B46D340D04020244F
:1001A000A21A91400843194610BD03460B439B0712
:1001B00003D009E008C9121F08C0042AFAD203E0DC
:1001C0000B780370401C491C521EF9D27047D2B202
:1001D00001E00270401C491EFBD270470022F6E786
:1001E00010B513460A4604461946FFF7F0FF2046AD
:1001F00010BD0321001D401E037812021A43491E40
:10020000F9D510467047F0B51FB40646002082B0FD
:1002100005464024019100901BE0019922460F46BB
:100220003046FFF7B1FF049A059B801A994110D31D
:1002300010461946224600F029F8361A8F410197D8
:10024000224601200021009F00F020F838184D417F
:1002500000902046641E0028DFDC019B00982946A0
:10026000324607B0F0BD0000064C0125064E05E001
:10027000E36807CC2B430C3C98471034B442F7D3C7
:10028000FFF71CFFA0570008C057000810B5202A30
:1002900004DB0146203A9140002010BD914020230C
:1002A0009C1A0346E3401943904010BDF0B51C4C26
:1002B000A0684007C00F31D1206C1B4D82B2194895
:1002C0001A4903690120DE07002E02D08A822846DF
:1002D0001AE09D4306D0164D9D430ED0154D9D430B
:1002E0000ED011E00A83154B134815499A4201D2EA
:1002F000012200E000220A6006E00A84114803E0BF
:100300004A84114A528BCA834103490BA162A168F6
:100310000E4A1140091DA160024908610020F0BD8C
:100320000024014000000020000100208C1000206B
:100330000000014000000244000001C098080000D5
:10034000D0000020000002C4A0F7FF1FE8FFFF7FDD
:10035000F0B51E4F85B03D691D4C6D1C3D61266892
:10036000A468029400966C466580019021816281A8
:100370000393386A01011748091800220B461046FA
:100380001C5CFF2C04D1401C1028F9D3002A17D084
:100390001022684600F012F9386AF861401C386291
:1003A0000001012109031030884201D90020386280
:1003B000F8680949401CF8604863002005B0F0BDAA
:1003C0001022684604F0CEF9E6E70000AC000020F9
:1003D0003857000800D000084C100020002911D028
:1003E0008268521882604368934200DCD21A00236C
:1003F0008361C368934201D1012343618260026932
:10040000521802610846704710B500231A4605E0ED
:10041000845C2407240FE318DBB2521C8A42F7DB0A
:100420001807000F10BD0000F0B50020174D012780
:10043000144B154C3F03E86017E0625A144EB24269
:1004400012D1EA680919521CEA604A882E69B24240
:1004500005D92A61E8614A686A61421C2A624988B2
:10046000994201D20B46A861401C0101B942E4D374
:10047000286A00011030B84201D900202862E868DB
:10048000F0BD0000FFC99A3B00D00008AC0000207E
:10049000AA55000010B50421054800F0B0F8054841
:1004A00000218161C1610161C1600162084610BD26
:1004B00000D00008AC00002070B5234DE86A401C55
:1004C000E862224C20688006C00F11D02868296B92
:1004D00040182860296B28465830064600F058F826
:1004E00020206060B06900280AD00020286368726C
:1004F00020688005C00F02D001204002606070BDFE
:10050000304600F011FA12494A78A3585B085B00A4
:10051000A350F36832684E78D2180C4B0C33F2506B
:100520000A4B4A781B1DD658360C36040643D65063
:100530004978625801231A4362502863054881684C
:10054000802211438160D3E7740200200000024042
:1005500080570008003801400B49C86A401CC86237
:100560000A4802689204D20F05D001225203426069
:1005700000220A634A7201688903C90F02D001216F
:100580004904416070470000080300200000024059
:1005900010B5002910D0C26843685218934200DC9D
:1005A000D21A00234361C2608468944204D10122BC
:1005B00082618360C360C361084610BDF0B585B039
:1005C00016460D46074600F00FFB01200290002062
:1005D0000090019503A9684600F06EFA00247608A1
:1005E00007E060003A5A41190023012000F0BEFAEA
:1005F000641CA642F5D800F0AFFA05B0F0BD7FB597
:100600000D46044600F0F0FA00206A4631C203A904
:10061000684600F051FA00F09FFA04B070BD000087
:1006200006490020C861064801690422114301619E
:10063000016940221143016170470000F01600205B
:1006400000200240064A0021D16106490A690223BE
:100650001A430A61486108694022104308617047E3
:10066000F01600200020024010B5054B0022DA6190
:10067000044A1369012423431361018010BD000063
:10068000F01600200020024010B50B4A0020D1686F
:10069000CB060A4904D5C86902231843C861102053
:1006A000D3685B0705D5CB6901242343CB610421C3
:1006B0000843D06010BD000000200240F01600206A
:1006C00070B5044600F0A2FA0546104E0AE0601C20
:1006D00008D0002C04D000F099FA401BA04201D9A8
:1006E000032070BDF068C007F1D1F068800601D525
:1006F0002020F060F068C00602D4F068400703D5FF
:10070000FFF7C2FF012070BD002070BD0020024035
:1007100010B50E4C0020207220710D480078002882
:1007200000D10120A070E0700120C0020921C9069B
:10073000886288620749802088620A2000F0AEF94A
:1007400000F096F96061002010BD00001400002048
:100750007300002000140048FEB5394D0121490204
:10076000284600F044FC00900120019040213548CB
:1007700000F03DFC044601210920C902C00600F03A
:1007800036FC4021284600F032FC00262E4D002881
:100790000BD0002013212D4A4901EF7803E01318F4
:1007A0005B181E75401CB842F9DB0098002802D186
:1007B00000F05EF9686128690127002814D10098CB
:1007C000002811D000F054F96969401A2049884284
:1007D0000ADBF9020922D20691617D21C9002F614D
:1007E000FFF798FC1B494884002C06D1E8680028D4
:1007F00003D01948018DC18406850198002817D0BF
:10080000002C17D0E86800280AD12F716E711348A8
:10081000026840218A4302606E7102680A430260E6
:10082000287A002808D12879002805D12F7102E004
:10083000002C01D12E716E71EC600020FEBD000015
:10084000000400480014004814000020CC0A0020D6
:10085000102700000C0D00200C1200200038004072
:100860000A07120F01219140014201D00120704777
:10087000002070470A07120F01219140014201D068
:100880000120704700207047F8B50B051B0E254C62
:100890005B001C1909239B01E31800930523DB016E
:1008A000E618012307469B020A07E5180020120FED
:1008B0003B0003F091FF09060A0E12191D21282F93
:1008C0002E00FF2928D800981BE0FF2924D8009883
:1008D00008E0FF2920D8B08A18E080291CD20F2018
:1008E00080012018808E11E0802915D2A88A0DE0A1
:1008F000402911D2B08E09E040290DD20B20800191
:100900000EE0808A02E0802906D2A88E1146FFF709
:10091000A7FFF8BD802901D30020F8BD1120800178
:100920002018EEE7CC0A0020C1688268914201DA03
:10093000501A7047914202DC4269002A02D0406896
:10094000401A704780690028FBD000207047C268B9
:100950008168914201DA501A7047914202DC826943
:10096000002A02D04068401A704740690028FBD036
:100970000020704706490122896912030818010105
:10098000914201D3FF3801380249000140187047F5
:10099000AC00002000D00008F0B5334C4B001C190F
:1009A00011239B01E518152302469B010020E31843
:1009B000892A25D00EDC2C4F2C4B4E00F619F61848
:1009C000803A130003F008FF091F1F152125292E67
:1009D000333A15008D2A3FD00CDC8A2A33D08B2A7B
:1009E00035D08C2A05D140293ADA0B208001201815
:1009F000808EF0BD992A03D0A12A01D0FE2AF8D119
:100A000080292DDA2EE00846F0BD102928DAB08AB8
:100A1000F0BD102924DAB08EF0BD102920DA0520AF
:100A2000C00108E008291BDA0F208001DFE7082950
:100A300016DA012080022018808AF0BD80290FDAA2
:100A40003420285EF0BD80290ADAA88AF0BD40294A
:100A500006DA0D208001CAE7402901DAA88EF0BD30
:100A60000020F0BD988EF0BDCC0A002040020000AE
:100A700010B5074A5068074B99695468A04201D0E5
:100A800050689969044A51430914401A10BD000086
:100A90003800002000E000E05505000031B500F00E
:100AA000B5F8009C0546601C00D0641C00F0AEF850
:100AB000401BA042FAD338BDF8B5054623480F467F
:100AC000017E012601290BD0012101762868204CE6
:100AD000012807D02046FFF7F3FD002813D030E0AF
:100AE0000220F8BD2046FFF7EBFD002829D1FFF7D3
:100AF00097FD2046FFF7E4FD0646164801690422EB
:100B0000914301611DE00020C04338606C6812E031
:100B10002046FFF797FD0E48FFF7D2FD06460D4829
:100B20000169022291430161002E01D03C6008E07E
:100B3000012080022418A868696880024018A04239
:100B4000E6D80248002101763046F8BDF0160020B4
:100B500050C3000000200240034801698022114375
:100B6000016100207047000000200240F0B51FB472
:100B700005461A480024017E16461F46012907D063
:100B8000012101761648FFF79BFD002803D021E0E4
:100B9000022005B0F0BD012D1AD0022D18D0042579
:100BA00016E0220130463946FFF7EEFA81B201988D
:100BB00062001018FFF758FD0948FFF781FD094949
:100BC0000A69520852000A61002803D1641CE4B289
:100BD000AC42E6D3014900220A76DAE7F01600209B
:100BE00050C300000020024005480169090605D5F0
:100BF000044941600449416000207047012070476A
:100C00000020024023016745AB89EFCD0148006811
:100C1000704700001001002002480168491C016073
:100C2000704700001001002010B50648016810222E
:100C300011430160002000F007F800F017F80020D1
:100C400010BD00000020024010B5044600F040F93D
:100C50007D21C900FFF748FA00F080FB0022214601
:100C6000501E00F025F8002010BD000008B50F4808
:100C70008169012211438161816911400091C2693A
:100C800001040A43C261C069002208400090114675
:100C9000501F00F00DF800221146901E00F008F8D9
:100CA00000221146501E00F003F808BD001002405B
:100CB00010B502F037FA10BDF8B504460068364D9D
:100CC000C00354D5E8690026C00007D4E8692904A8
:100CD0000843E861E8690840012600902F48016850
:100CE000C90511D4014608688A1510430860FFF74A
:100CF0008DFF074604E0FFF789FFC01B642823D857
:100D000026480068C005F6D5286A03210902084074
:100D10001FD062680A4082421BD0286A2A6A884330
:100D2000012109040A432A622A6A8A432A62286244
:100D3000C0070ED0FFF76AFF074607E0FFF766FF20
:100D4000C11B1748814201D90320F8BD286A8007DA
:100D5000F4D5286A032109028843616808432862A0
:100D6000002E04D0E869012109078843E861207852
:100D7000C00705D0286BA16880088000084328635D
:100D80002078800605D5286B10218843E168084348
:100D900028630020F8BD00000010024000700040F1
:100DA00088130000F8B5044644480E460068C007A2
:100DB000C00FB0420AD24148016849084900314396
:100DC00001600068C007C00FB0425CD120783C4F82
:100DD000800705D57868F0218843A16808437860CA
:100DE0002078C0073FD06068012813D039680228F6
:100DF00013D08907002946DA7968890889000143F8
:100E00007960FFF703FF0546606801280DD00228CE
:100E100017D024E039688903ECE78901EAE7FFF796
:100E2000F5FE411B2748814217D878680007800FDC
:100E30000128F4D117E0FFF7E9FE411B2148814268
:100E40000BD878680007800F0228F4D10BE0FFF779
:100E5000DDFE411B1B48814201D90320F8BD7868A3
:100E60000007800FF3D115480168C907C90FB142C7
:100E70000BD9016849084900314301600068C00787
:100E8000C00FB04201D00120F8BD2078400706D540
:100E90007868072109028843E1680843786000F018
:100EA0001DF87968084A0906090F515CC8400749CE
:100EB00008600020FFF7C8FE0020F8BD00200240B7
:100EC0000010024088130000855700080C01002024
:100ED00001480068704700000C01002010B513A005
:100EE0000FC888B06C460FC414A00FC80FC4174BAE
:100EF0005A680C2011460140154804290FD00829D2
:100F00000DD19102090F6C46645CD96A04AB0907E4
:100F1000090F595CD20304D5FFF7E6F8604308B027
:100F200010BD0C4920464843F9E7000002030405C0
:100F3000060708090A0B0C0D0E0F1010010203041E
:100F400005060708090A0B0C0D0E0F1000100240D1
:100F500000127A0000093D000422044904280869AF
:100F600002D09043086170471043FBE700E000E0C7
:100F7000154801686431016014480168491C01602A
:100F800013490868401C08601249134AC868401C8D
:100F9000C860904216DB0020C86010488169491C77
:100FA00081610169491C01614169491C41610C4928
:100FB000088B002806D0401E80B20883782801D90B
:100FC00078200883704700003C0000203400002097
:100FD00084000020DC000020102700004C100020BE
:100FE0004012002010B5FFF7C3FF10BDFEE70069F7
:100FF000814301D00020704701207047704770473F
:10100000332E303000000000FEB504460078D04D8D
:10101000C00746D068680007800F012807D06868BD
:101020000007800F022809D16868C00306D5286828
:10103000800336D5606800287ED032E001216068E8
:10104000090401280AD08A00002801D005280FD001
:101050002868884328602868904301E0286808438E
:1010600028606068002810D0FFF7D0FD064608E031
:10107000286810432860F1E7FFF7C8FD801B64284B
:101080006FD828688003F7D50BE0FFF7BFFD064651
:1010900004E0FFF7BBFD801B6428F1D828688003BB
:1010A000F7D420780126800700283BDA686800071B
:1010B000800F07D068680007800F022809D1686890
:1010C000C00306D42868800715D5E068012833D10D
:1010D00011E0E0680028286815D030432860FFF749
:1010E00095FD074604E0FFF791FDC01B0228C7D815
:1010F00028688007F7D52868F82188432169C90046
:10110000084328600EE0400840002860FFF77EFD9D
:10111000074604E0FFF77AFDC01B0228B0D8286814
:101120008007F7D42078000724D5E0690028686A92
:1011300010D03043686200E007E1FFF767FD074623
:1011400004E0FFF763FDC01B022899D8686A800796
:10115000F7D50FE0400840006862FFF757FD0746EB
:1011600005E09DE0FFF752FDC01B022888D8686AA1
:101170008007F7D4207804274007002860DA002091
:101180000190E869C00008D4E969B8060143E96143
:10119000E96901400120009101906E480168C9058C
:1011A00011D40168821511430160FFF72FFD0090F3
:1011B00005E0FFF72BFD0099401A642870D86548B8
:1011C0000068C005F5D5A06801280AD0002801D024
:1011D000052810D0286A400840002862286AB843D1
:1011E00001E0286A30432862A068002812D0FFF787
:1011F0000DFD00900AE0286A38432862F1E7FFF706
:1012000005FD0099411A5448814249D8286A80074F
:10121000F5D50DE0FFF7FAFC009006E0FFF7F6FCCD
:101220000099411A4C4881423AD8286A8007F5D47F
:101230000198002804D0E969012000078143E96191
:101240002078C00635D5606901280CD0401D686B38
:1012500023D038436863686B400840006863FFF739
:10126000D5FC064622E0686B38436863686B304300
:101270006863FFF7CBFC064604E0FFF7C7FC801B62
:1012800002285BD8686B8007F7D5686BF821884324
:10129000A169C900084368630BE0B8436863F4E7D9
:1012A0004CE0FFF7B3FC801B022847D8686B80072F
:1012B000F7D4206A002846D069680907890F0229F7
:1012C00043D001273F060228286805D0B84328608C
:1012D000FFF79CFC044633E0B8432860FFF796FC18
:1012E000064604E0FFF792FC801B022826D82868F7
:1012F0008001F7D4E86AE16A000900010843E86266
:10130000616AA06A084369683D2212049143084358
:101310006860286838432860FFF778FC044604E0DA
:10132000FFF774FC001B022808D828688001F7D555
:1013300009E0FFF76BFC001B022801D90320FEBD6A
:1013400028688001F5D40020FEBD0120FEBD00000C
:10135000001002400070004088130000094910B5D9
:10136000401E884201D9012010BD074C6061032155
:10137000081F01F0D7FE0020A06107202061002097
:1013800010BD0000FFFFFF0000E000E010B50021ED
:101390000F4A0846516043009B18401C1981FF28E2
:1013A000F9DD002005230B4ADB014400A418E418F2
:1013B000401CA1821028F8DB002011239B0144006F
:1013C000A418E418401CA186FF28F8DD002010BDF9
:1013D000E4140020CC0A002010B5402802DB0020D5
:1013E000C04310BD10221143C200094B4000D21867
:1013F000C01858240D23A1529B010021C3189986BF
:10140000E300C0188186034800685065084610BD97
:10141000CC0A00201001002070B504461E4638306A
:10142000049D03F0ADFC20462A463146583003F0B7
:10143000A7FC002070BD000070B5104D06460146A7
:101440002846FEF767FE0E4C2061FFF741FD294656
:10145000FEF74AFEA0600B48314600680546FEF7DD
:1014600043FEE0602A46002307480F21FEF766FE90
:101470002080206964306060002070BD40420F0011
:10148000380000200C01002000004042034610B547
:101490000020024602E09C5C6040521C8A42FADB5B
:1014A00010BD0000F8B508460E460978552901D050
:1014B000252903D0012A01DD461C521E344F602429
:1014C000797933786143334C0919334C252B30D06B
:1014D000A3685B1CA360CB695B1CCB61B978002956
:1014E0000FD0F97800290FD001292C4913D01B23E4
:1014F0009B01C9180A7501462948FEF756FE0020CF
:10150000F8700020C043F8BD2549264B55390A75AF
:101510000146224807E035235B01C9180A750146D8
:10152000204B1E482033C018FEF73FFEF878401CC1
:10153000E6E74579802D06DDE068401CE060086A3A
:10154000401C0862DDE72B4608339A4208D2086A3D
:10155000401C0862E068401CE0600220C043F8BD07
:10156000A91DFFF793FF7119897981420DD0206978
:10157000401C206179796020414306480818416A7F
:10158000491C41620320C043F8BD0020F8BD0000A3
:1015900068000020BC05002088030020CC0A002041
:1015A000A111002095060000F8B50E46044625203E
:1015B000069F079D089920706270A670E3702771DE
:1015C0002F46002008376619372B1AD009DC1A4637
:1015D000303A130003F000F90726151526262617C2
:1015E0002600612B0DD006DC382B0AD0412B08D009
:1015F000422B17D105E0622B03D0632B01D0642B63
:1016000010D1657102E06571002D03D02A46A01D3E
:10161000FEF7CBFDA91D2046FFF738FFB0710D2066
:10162000F0713846F8BD0000F1B584B0FFF7EEFA6E
:101630000446FFF71DFA484DE979002906D0297ABA
:10164000002903D0E968411A322905D8E9687D22CA
:10165000411AD200914253D9297A404A404E00297A
:1016600051D06B79602701217B43F1506421516097
:101670006979491CC9B26971EA7A914208D9A96AA3
:10168000411AE962A862A979491CA971012169710D
:101690003449098A344B6A7934499F5C0F709B182E
:1016A0005B784B7060235343F35C8B700027CF70E3
:1016B0000C71230A4B71230C8B71230ECB71E860E4
:1016C000AB790820019028480093029141233946C4
:1016D0001030FFF769FF244902461031049802F0E8
:1016E000D3FB68796021484380194168491C4160F7
:1016F000C268E9688A1A4263C1606C63EF712F7235
:10170000002005B0F0BD696A491C696218494B6840
:101710005B1C4B60697960238E4659438C4689195E
:101720000B695B1C0B614B695B1C4B61EF79002FF4
:1017300002D18F6A7F1C8F628F69BB4200D98B6197
:10174000032B95D900216346F150C8239360064BC3
:101750007246103B99548BE7680000204C10002023
:10176000BC05002040120020AC040020BC08002072
:1017700088030020F7B5087886B00C46552801D0BC
:10178000252802D0012A00DD4C1C424E6279707976
:1017900060210490484340494518A868401CA8604F
:1017A00008468038039031460B6BC968E778591AB0
:1017B0003346A0789B69303F00933B0003F00CF860
:1017C00013420B17424242294242424242424242A3
:1017D00042422C4542003149A3790B542179A01D86
:1017E00032230192009102900021049A22E071615B
:1017F000009A914200DDB161284AA3791354002078
:10180000E9626861286B884200D229630120307246
:1018100018E00120F07115E02048A1790170103026
:101820000078A0712179A01D0192009102904223BD
:10183000317900220398FFF7B7FE02460399069814
:1018400002F022FB002009B0F0BD7161009A9142C4
:1018500000DDB161114BA2791A54114B18180923FC
:101860009B01C018C2740F48008A0020E9626861B9
:10187000286B884200D229632046677A0A30FEF737
:10188000B8FC617B0002000A09060843B900691828
:101890008863BBE768000020BC0500209C04002092
:1018A000CC0A002040120020F7B515460C46FFF781
:1018B000DFF81A4E306321780020552903D1012D1D
:1018C00001DD641C6D1E317800290FD00127F771EE
:1018D0002A4621460098FFF7E5FD002805D137721A
:1018E0002A4621460098FFF745FFFEBD7178002982
:1018F000FBD00B4E2A46B06B2146401CB0630098CB
:1019000000F012F80028F0D106482A4640683065F9
:101910002146009800F078F8FEBD00006800002025
:10192000BC0500204C100020F0B508460D46097893
:10193000552901D0252903D0012A01DD451C521E5D
:10194000297800231A4FDB431A4C252906D0A068BA
:10195000401CA060386C401C386409E014496E7962
:10196000896C491C802E05DDE068401CE060B9648C
:101970001846F0BD334608339A4206D2B964E0688F
:10198000401CE0600220C043F0BDB11DFFF77EFDAA
:10199000A9198979814208D02069401C2061F86C1E
:1019A000401CF8640320C043F0BD0020F0BD0000DF
:1019B000BC0500208803002070B5FFF759F80F4BD5
:1019C0001A695D7A7D24A4010D49002D03D0002001
:1019D0004C6058720FE00B4D861AAE4202D90122BC
:1019E0008C6004E05219904205D902228C608A630F
:1019F000C86318690864002070BD000068000020FA
:101A00004C100020E02E0000F7B5524884B0026868
:101A1000521C02604A794B784F48504D03904E4C0F
:101A200028798034834208D0FF2B06D0606C401C9C
:101A300060640020C04307B0F0BD834201D0FF2B9B
:101A400079D1464D2B6B00932B6101236B72424B76
:101A5000CF78903B8D1D1E78372F79D007DC303F33
:101A60003B0002F0B9FE0675137575752275612F7E
:101A70006ED004DC382F6BD0412F69D125E0622F66
:101A800066D0632F64D0642F62D155E0324B8F79DA
:101A9000A03B1F708E71314B009E1E6109796F460D
:101AA00026C732230022014607E0002009793623A9
:101AB000009101900246029001210398FFF774FD06
:101AC0000246E06B401CE06331E0234B8F79A03B82
:101AD0001F70CF7A8B7A3F02DB19204FFB61BB7AF4
:101AE0008E711D4C9E0080344B723419268F8E727D
:101AF000268F5B1C360ACE72A66BDBB2360C0E73D9
:101B0000A46B240E4C73BB720A2B01D30023BB724F
:101B100009796C4626C40146422300220398FFF748
:101B200043FD02460C488030C16B491CC1630399D8
:101B3000049802F0A9F90BE0CA7988791202821898
:101B4000087A497A00040906401811180348C1614F
:101B5000002070E7880300203C050020680000207A
:101B6000034610B50020024602E09C5C6040521C17
:101B70008A42FADB10BD30B50D4608460978144696
:101B8000252901D0012030BD062C01D2032030BD13
:101B9000611EFFF7E5FF29192039C97F814201D075
:101BA000042030BD002030BDF8B51E460B46552739
:101BB000069D0799077043708270C67004460571D0
:101BC0002A46401DFEF7F1FA691D2046FFF7C8FFBF
:101BD000014660194171A81D052E02DA002E00D1C0
:101BE0000020F8BDFEB516460F460546FFF7C3FFB9
:101BF000040014D0684604720420009002A90B4827
:101C000001910278401E0178EE230948FFF7CCFFCE
:101C100002460749284602F037F92046FEBD324603
:101C20003946284600F006F8FEBD0000A10000205D
:101C30004C090020F7B54F7886B00C46FE48426844
:101C40008260421C15788E782D0936072D01360FDB
:101C50000B7935431570F94A029200780490874257
:101C600001D0FF2F77D12146E6780931F4488C4620
:101C7000332E72D028DCF349182E09686CD012DCA0
:101C8000072E20D008DC002E65D0012E3ED0032E7A
:101C900041D0052E7ED160E0112EF5D0162E7AD0DF
:101CA000172EF7D13EE2232EEED006DC192E73D08C
:101CB000212E72D0222EEDD19EE1242EE4D0312EA1
:101CC0004BD0322EE6D1BEE0582E67D012DC542E17
:101CD00072D008DC342E70D04F2E6FD0502E6ED0C4
:101CE000532ED7D172E2552E6AD0562E69D0572E78
:101CF000D0D168E2304663380421030002F06CFD65
:101D000009EFEEED171D4A104A154A00641D0093B5
:101D10000194012355E2CC49182003E03946CAE278
:101D2000CA490C200191009005E0C948F5E1C84975
:101D300010395020F6E7334643E2E1790020BF4AEC
:101D400003E023185B7A1354401C8842F9DBBB483C
:101D500002F0A4FCA2E079E2EEE1A279617912023C
:101D60008918E27989B2882B2CD0892B2ED08A2B26
:101D700030D0832B33D0842B36D0852B39D0862B93
:101D80003CD0872B3FD08B2B42D08C2B45D0FE2BC9
:101D90001CD004E09AE2AEE1EFE1CEE06BE2A92BC9
:101DA00040D0B32B42D0992B43D0A12B46D0A3488F
:101DB00010384018009265E21FE244E0FBE1F6E1D2
:101DC00045E24EE249000918A2483AE049000918E4
:101DD000A14836E0490009189E48203831E0490002
:101DE0000918952080002CE0490009189D208000EA
:101DF00027E049000918A520800022E049000918C1
:101E0000FD2080001DE0490009189248603818E064
:101E100049000918DD20800013E049000918BD20A1
:101E200080000EE0490009188C480AE049008C48FF
:101E300007E08C4849000818001DBBE74900012055
:101E4000C0060818B6E7A279617912028918E2790A
:101E500089B2882B2AD0892B2CD08A2B2ED0832B89
:101E600031D0842B34D0852B3AD0862B3DD0872B94
:101E700040D08B2B43D08C2B46D0FE2B4AD0A92BA5
:101E80004CD0B32B4ED0992B4FD0A12B50D06B48B8
:101E90001038401800226146FEF787F900200090B4
:101EA00001906548E378401C027837E7490009183B
:101EB000684840E04900091867483CE049000918B3
:101EC0006448203837E0490009189520800032E046
:101ED000490009189D2080002DE0E3E1D6E1D3E11F
:101EE00049000918A520800025E049000918FD20B7
:101EF000800020E049000918564860381BE049007E
:101F00000918DD20800003E049000918BD20800089
:101F10000818BFE7490009184F48F9E749000918B0
:101F20004E48F5E749004E48F2E749004D4802E0C7
:101F300049000120C0060818ADE7A27961791202B4
:101F400089180922920189B2002B0ED0012B16D0DC
:101F5000022B1AD0032B25D0042B31D0052B35D0E2
:101F6000062B33D0082B3FD007E00B095B00181875
:101F70008018828A1DE001202EE000202CE00B0951
:101F80005B0018188018808E05E00A0952001018AE
:101F90000522D2012DE00A07120F012191400840CD
:101FA000E9D119E00A09520010180F229201801895
:101FB000828E0907090F012088400242DDD0DAE74E
:101FC0000A09520010180122920212E0C9000818F2
:101FD0004030007E4006C00F69460873012003A907
:101FE000212301910090ECE00A09520010181122FF
:101FF00092018018808ACEE7A2796179120289184D
:1020000089B2002B33D0012B3AD0022B41D0032BC5
:1020100048D0042B4FD04022052B54D0062B52D051
:10202000072B5BD00020694608730020009002480F
:1020300003A90191401C17E0A00000204C090020DA
:10204000CC0A0020E4140020A0560008ACF7FF1FC3
:10205000107C000874040000740500007406000081
:10206000BC0500204C0A00200278222356E60B070C
:102070000909490009181B0F9520E279800035E015
:102080000B070909490009181B0F9D20E279800000
:102090002CE00B070909490009181B0FA520E2795C
:1020A000800023E00B070909490009181B0FFD20D8
:1020B000E27980001AE00B0709091B0F4900091893
:1020C000E279884812E0C90008184030018B91433A
:1020D000E279D207520E11430183A6E70B070909E3
:1020E000490009187F48E2791B0F4030081819464B
:1020F00001F0EEFE99E7A179607909024018E179D3
:10210000794A80B2002B0AD0784C012B03D0784B4F
:102110009B8A002B03D0400000190091B2E04000E0
:102120008018FAE77348002901D0002101600020DF
:1021300000901723019044E06E48002901D000214F
:102140000160A17960790902401885B2E279002026
:10215000694903E02618767A0E54401C9042F9DB58
:102160006549284602F0A8FA002009340090019041
:102170006248039402781823D0E5A17960790902B6
:1021800041185B48C182818A00290ED000218182DA
:10219000574801F003FE57480121016000200090DC
:1021A0000190564819230278B8E50121EFE750481D
:1021B0000383002002E04E49002008830090019034
:1021C000E3782A46AAE54A492020ABE5A17960795F
:1021D000090240184A4980B20A18E179121D78288C
:1021E00001D3002105E00B18782B02D97821081AB9
:1021F00081B2C8B2019200909DE5A179607909028F
:1022000040183F4980B20B18E2791B1D782801D392
:10221000002205E01118782902D97821081A82B223
:1022200061461846FDF7C1FF002000900190334839
:10223000E378027839460298FFF7B6FC0246029925
:10224000069801F021FE2E4802F056FA3BE02C4899
:1022500002F052FA0020009001902848552302789D
:102260005CE5234801F09AFD00200090019023488E
:102270005623027852E5032109022248FDF7AEFFFA
:1022800000200090019056E51F4846E7A17960794B
:1022900009024018E17980B20D01FEF76BFBE9B24B
:1022A0000091FDE5FEF7F6F800200090019013483C
:1022B0006523027832E50298FFF776FC0246029920
:1022C000069801F0E1FD002009B0F0BD022069464A
:1022D000087303A901200191EE232A460090049976
:1022E000E9E70000140400000080000800A00008D6
:1022F00040120020E41400204C090020A10000201E
:102300004C0A0020BC0500208010002070B5FEF7AC
:102310008BF8154800F066FA144D154C6869A061F9
:102320001148816861618188491C81808088E060F2
:102330000D4801F033FD2868206368686063A86871
:10234000A06301220B4B1146A069FEF701F8E86873
:102350002064A8696064E869A0642869E064286A68
:102360002065002070BD000040120020AC0000205D
:102370004C1000203930000008B504494A69024376
:102380004A6149690140009108BD00000010024007
:1023900008B50449CA690243CA61C969014000918C
:1023A00008BD00000010024008B504498A690243D4
:1023B0008A6189690140009108BD00000010024057
:1023C00070B5094E04467618203E049D0C34F17F0A
:1023D0000830102D03D00A50F07F035170BD0A5110
:1023E000F17F0B5070BD00009A520008044A51184A
:1023F0002039C97F425852085200425070470000AD
:102400009A520008044A51182039C97F42580123C2
:102410001A434250704700009A520008044A51186B
:102420002039C97F425802231A43425070470000A6
:102430009A520008054B10B559182039C97F4358E6
:1024400003242403A3431343435010BD84520008C4
:10245000054B59182039C97F001D0B581B0C1B0454
:1024600013430B50704700009A520008054B10B5FB
:1024700059182039C97F4358034C23401343435014
:1024800010BD000084520008EFBFFFFF054B10B5E0
:1024900059182039C97F43588024A343134343501C
:1024A00010BD000084520008054B10B559182039A2
:1024B000C97F43580324A402A3431343435010BDD0
:1024C00084520008054B10B559182039C97F43586C
:1024D0002024A3431343435010BD0000845200083E
:1024E000054B10B559182039C97F43584024A343E0
:1024F0001343435010BD000084520008054B10B533
:1025000059182039C97F435803242402A343134395
:10251000435010BD84520008F0B500233CE0012474
:102520009C40224037D04F680668144654436500EB
:102530006519AE4367433E4306604E68012E01D0E5
:10254000022E05D18F6886686743AE433E4386609E
:102550000F69C668AE4325467D432E43C6604D686D
:10256000022D18D14D69FF2A09D8066A54435443F5
:102570002201121B96436C43264306620BE0140AA9
:1025800022466243624362431401A61A446A6A43C4
:10259000B443144344625B1C0A681446DC40BED159
:1025A0004A68012A01D0022A06D10A68C96843682C
:1025B00093434A43134343600120F0BD10B50446E2
:1025C00001F0B6FA206001F099FA606001F0A4FA17
:1025D000A06010BD014610B5002000290FD1104A9F
:1025E000116B8907890F01290AD0022911D003290B
:1025F00009D001F09DFA01F081FA01F08DFA10BDC9
:1026000001F096FA10BD11688907C90FFAD0054884
:1026100010BD116A8907C90FFAD00120C00310BD8F
:102620000010024000127A0010B5036800225B0619
:10263000DB0F25D10CC98C681A434B6823431A431E
:10264000CB681A430B691A434B691A438B691A43C7
:1026500003680C4C23401A43026042680A4B1A403C
:10266000CB681B0C1A430B681A43426001238A692A
:102670005B0308399A4202D1898C89B20161012237
:10268000104610BD4000FFFFFBF0FFFFF0B50268F1
:10269000194B1A4C984201D0A04203D17025AA438D
:1026A0004D682A43164D174E174F98420AD0A04244
:1026B00008D0164CA04205D0A84203D0B04201D0A9
:1026C000B84204D103242402A243CC68224302600E
:1026D0008A68C2620A888262984205D0A84203D002
:1026E000B04201D0B84201D1097C016341690122A5
:1026F000114341611046F0BD002C01400004004030
:1027000000400140004401400048014000200040DA
:1027100041680122D20291434160816808229143BD
:1027200081607047FEB5044600680D460026C0076C
:10273000C00F43D1E9686868AA6908432969114351
:10274000084321681E4A114008432060A868616858
:10275000032212039143014361606869A168121169
:1027600091430143A1601748844203D10020FFF741
:1027700031FF06E01448844220D16846FFF71EFF6F
:10278000029800281AD02968002917D00126AA69C2
:10279000F3039A420CD140004A088018FDF7A4FCCC
:1027A0000A4980B201400007420F0A43E26005E097
:1027B0004A081018FDF798FC80B2E0603046FEBD74
:1027C000F369FFFF0038014000440040F0FF0000C3
:1027D00010B580220249FDF7E8FC002010BD000082
:1027E000B8560008F0B5134A00215514124C134F87
:1027F0000CE0D65ABE4208D19B185B886668B3428B
:1028000003D90AC44B1C2360083C491C4B01AB4252
:10281000EFD32168002904DB49018918202201F047
:10282000BDF9A06840012030A84201D90020A06075
:102830000020F0BD00C80008AC000020AA55000030
:102840001FB50B46024604A1684601F0B1FF0146E0
:10285000684601F031F91FBD201B5B25643B2564F0
:102860004800000010B50120FFF786FD00210A2076
:1028700000F036FC0A2000F029FC00210B2000F0BB
:102880002FFC0B2000F022FC10BD0000F0B5012051
:1028900087B04004FFF770FD01208004FFF76CFD56
:1028A0000120C004FFF768FD01208005FFF764FDEB
:1028B0000126C020002403256A46049631C2092758
:1028C000FF0669463846FFF727FE8020694631C17A
:1028D000694638460494FFF71FFE932000010090DC
:1028E000039469460196029504943846FFF714FE56
:1028F0003002B86168026A46049631C269463846B9
:10290000FFF70AFE29486A46049631C269462848FC
:10291000FFF702FE2748009003946946019602954E
:1029200004942348FFF7F8FD072040030090029429
:1029300003946946019604941F48FFF7EDFDF020CB
:102940006A46049631C269463846FFF7E5FD300213
:10295000B86140006A46049631C269461448FFF7E0
:10296000DBFD40206A46049631C269461348FFF7F2
:10297000D3FDF00200906946019602950494384612
:10298000FFF7CAFD802000906946019602950494E5
:102990000A48FFF7C1FD40206A46049631C26946E5
:1029A0000348FFF7B9FD07B0F0BD000007040000C1
:1029B00000040048C0FC0000000800480014004863
:1029C0000848074901600849016004214160074A3D
:1029D0008260C1684907FCD1026105490160704706
:1029E000CCCC00000030004055550000FF0F000027
:1029F000AAAA0000F0B591B0282106A8FDF7EEFBC9
:102A000018216846FDF7EAFB01200003FFF7CCFC24
:102A100001208004FFF7B0FC0024082502260327CC
:102A2000039404946A460594E0C269462248FFF77D
:102A300073FD102069460394C1C1012004906946CA
:102A400005941D48FFF768FD2020039404946A460E
:102A50000594C1C269461848FFF75EFD00211920A0
:102A600000F03EFB192000F031FB07200002089027
:102A7000012006940A9040020B900994802007944C
:102A80000E940D9007200D4C0F900C9506A9204632
:102A9000FFF7CAFD60681021884360606068A84342
:102AA00060606068090288430843606020684021D4
:102AB0000843206011B0F0BD000400480030014020
:102AC00010B586B014216846FDF788FB1020FFF78B
:102AD0005FFC0021112000F003FB112000F0F6FA4A
:102AE0002F2069460880002001900848084C029079
:102AF0002046FFF7CBFD2068802188432060E068F6
:102B000001210843E06006B010BD0000E7030000AB
:102B10000010004070B501208EB08003FFF744FC28
:102B2000032040020790022008900320002409900F
:102B3000012509200A9407A90C950B94C006FFF7FC
:102B4000EBFC3A4E102202213046FFF78FFC0022A8
:102B500002213046FFF76EFC002202213046FFF7CB
:102B6000B1FC002202213046FFF7BAFC802202218C
:102B70003046FFF78BFC002202213046FFF7BEFCF7
:102B8000002202213046FFF78FFC0022032130464D
:102B9000FFF76CFC002203213046FFF74BFC0022BC
:102BA00003213046FFF78EFC002203213046FFF759
:102BB00097FC802203213046FFF768FC00220321A6
:102BC0003046FFF79BFC002203213046FFF76CFCE8
:102BD00000211B2000F084FA1B2000F077FA144833
:102BE0006946006800900194029403940594069449
:102BF0000C20104C04902046FFF794FD60682905D6
:102C0000084360606068490003225205904308430E
:102C10006060A06849120843A0602046FFF778FD75
:102C20002068284320600EB070BD00000000024004
:102C3000500000200038014070B58EB01C2168465D
:102C4000FDF7CCFA182107A8FDF7C8FA012464049F
:102C50002046FFF79DFB2046FFF78EFB0E200790D6
:102C600002200890032001250990002409200A95DC
:102C700007A90C950B94C006FFF74EFC414E10229D
:102C800004213046FFF7F2FB002204213046FFF713
:102C9000D1FB002204213046FFF714FC002204215E
:102CA0003046FFF71DFC802204213046FFF7EEFB83
:102CB000002204213046FFF721FC00220421304687
:102CC000FFF7F2FB002205213046FFF7CFFB002281
:102CD00005213046FFF7AEFB002205213046FFF705
:102CE000F1FB002205213046FFF7FAFB8022052187
:102CF0003046FFF7CBFB002205213046FFF7FEFBF5
:102D0000002205213046FFF7CFFB00211C2000F0F8
:102D1000E7F91C2000F0DAF9A61EFF21304600F08A
:102D2000DFF9304600F0D2F91748EE030068009052
:102D30000194029403940C2004AA51C2134C6946D6
:102D40002046FFF7EFFCA06821140843A060A068AC
:102D5000B0433043A06020681F21490588430843E1
:102D6000206020684911884308432060A068A114AE
:102D70000843A0602046FFF7CBFC20682843206072
:102D80000EB070BD0000024054000020004400401E
:102D900000B50846042A02D80020C04300BD0178CF
:102DA0007F2902D90120C04300BD41784906490E60
:102DB0001F2902D90220C04300BD114601F0AAFF1D
:102DC0000028F9D0042000BDF7B588B00F460A9A54
:102DD0000898FFF7DDFF0690002803D00020C043CD
:102DE0000BB0F0BDB6483A780078394682427DD1C2
:102DF0008C784A78CB78B98824024DBAB1491C4303
:102E000008704A7001200790200521070226000E55
:102E1000090F130001F0E0FC119E0A47859FB7D50A
:102E20009E9E9E9E9E9E9E9EE1F39E00E81DC00873
:102E3000A4490390887000202FE00020009001201A
:102E4000019002980027C00004901CE02005000EAD
:102E500042009D4821071218092080011018090F0F
:102E6000808EFDF707FD002803D0019900980843E4
:102E700000900198641C4006000E7F1CA4B20190D3
:102E8000082F03DA0498C019A842DFDB8D49029AA3
:102E900000988918C8700298401C039902908842D3
:102EA000CBDB761855E0E81DC00886490390887092
:102EB000002031E0002000900120019002980027BE
:102EC000C00004901EE02005000E42007E4821074D
:102ED0001218092080011018090F808AFDF7CAFC1A
:102EE000002805D001990098084300E0E5E0009033
:102EF0000198641C4006000E7F1CA4B20190082FAC
:102F000003DA0498C019A842DDDB6E49029A0098E2
:102F10008918C8700298401C039902908842C9DB46
:102F2000BFE7680067498446887000200EE02118DA
:102F30004A00654947005218112189015118898EAC
:102F4000604A0B0ABA18D3701171401CA842EEDB1C
:102F500017E0761C87E068005A4A8446907000208B
:102F60000DE021184B00584947005B1809218901E1
:102F70005918898ABF180B0AFB703971401CA84286
:102F8000EFDB6644E5E7002D12D0FF2212029542E6
:102F900007D142004C4812189D208000101800F004
:102FA0008FFF394647480A9AFDF7FFF80A9E7FE0EF
:102FB0004200454812189D208000101800F040FE85
:102FC000EFE738797979000208433F4962005218E7
:102FD0001121890151188886E3E7E81DC0083949A5
:102FE00003908870002030E03818C07900900120EC
:102FF0000190002005900298C00004901FE036E088
:103000002005000E42003048210712189D20090FAC
:1030100080001018009B019A1A4202D000F050FF65
:1030200001E000F00DFE0198641C4006000E0190C6
:103030000598A4B2401C0590082804DA0498059964
:103040004018A842DCDB0298401C03990290884299
:10305000CADB1C48B9788170F978C170397901717F
:1030600079794171361D0698002814D025E000209A
:103070000EE04100C919CA79097A12020A432118DF
:103080004B0011495B181121890159188A86401C8F
:10309000A842EEDBDDE70798002809D0B1B2094865
:1030A00001F038FE07498855000A89194870B61C96
:1030B00032460449089800F0E7FE002090E6000040
:1030C0000401002064140020CC0A0020C106C90EAF
:1030D00001208840014908607047000000E100E0DD
:1030E0008307FF22DB0E9A408907090E99400028CA
:1030F0000BDA0007000F0838830808489B001818EF
:10310000C36993430B43C3617047830804489B0022
:103110001818036893430B430360704700ED00E009
:1031200000E400E08307FF22DB0E9A408907090EC6
:10313000994000280BDA0007000F08388308084878
:103140009B001818C36993430B43C36170478308FE
:1031500004489B001818036893430B4303607047AF
:1031600000ED00E000E400E0F3B5074681B0002088
:1031700000903D78FF206E07EC08760FE40001F028
:103180000BFE802C01D20020FEBD324601265C4998
:103190005C48130001F020FB0805313539898D9119
:1031A000A1B057490978002903D0554949788C4284
:1031B00020D18188544F491C81803D70504D302171
:1031C000A87808437870E8780843B8703520F8701C
:1031D00004213846FDF718F93021084338710D20D5
:1031E0007871112001F0D8FD0621384600F016FE56
:1031F0006C702E704248067162E0C188491CC18023
:103200005EE00189491C01815AE00A78002A02D057
:103210004A78A24201D00E7152E042893849521CCC
:1032200042810020CA780EE04100C9194B788978A4
:103230001B010907090F5B1834490C1813214901B8
:1032400061180B75401C2E4C9042EDDB2E4A00207D
:1032500015702E4F0FE009213B1889015B18197D6D
:103260000D094100891830354D701B7D1B071B0F60
:1032700030338B70401CA1788842ECDB0806C00D0F
:10328000401CC1B22048FDF7BFF830210843A178A7
:103290001D4A49008A1850700D209070C91CC9B28F
:1032A000194800F0BBFD26710AE08189491C818123
:1032B00006E0C189491CC18102E0018A491C0182E2
:1032C00002980007C10E114809180920C00108180A
:1032D000818C491C81840098FEBD428A521C428226
:1032E0000878002897D04878A04294D10120C002E5
:1032F0000922D20690618EE7028B521C02838AE774
:10330000140000204C0F002014020020CC0A0020E2
:1033100010B501200449C006486004480168491CF2
:10332000016000F005F810BD00ED00E04C00002049
:1033300070B50E4801780024002905D004700C48AF
:1033400001780C48FFF710FF0B4DE86F00280BD0F9
:103350000A4E0B4902203268FEF7A6FA3460EC6789
:103360008021074801F012F970BD00002C000020F8
:103370002D00002054020020080300205C000020E3
:103380001C04002010B50648054B00780021403B86
:103390005A1840325478491C14700F29F8DB10BDBC
:1033A0000C0B002010B5084C084B01220221A0692B
:1033B000FCF7CEFF064800F0F1FCE069401CE0613C
:1033C000A0692062002010BD4C10002039300000A0
:1033D000401200200248C169491CC16100207047A9
:1033E0004C100020F3B5FA4D85B0286800286FD046
:1033F000686800281CD000220D21082000F080FD04
:1034000000221146082000F07BFD01221146082011
:1034100000F076FD00200146EE4A13184033401CB0
:1034200019701028F8DB00260121144640347BE295
:103430000122E1E7B2000598059B805CD7187A78F5
:10344000019201257B8800931B2873D012DC024671
:10345000030001F0C1F91B5C7272727272723E3E1F
:103460003E3E3E3E5C5C5CA7A7A73E3EBEBEBEBEE7
:10347000BEBE5C00342870D011DC01461C390B0044
:1034800001F0AAF918A7A7A7A7A7A7A7A7A7A7A763
:10349000454545454545454545454545F7453A2852
:1034A00073D008DC014635390B0001F095F905E2CF
:1034B0006E56E26E3000DC2804D004DC3B28EFD0EE
:1034C000C82824D120E1DD28FCD0FA28F9D11BE15D
:1034D00033E2D01F030001F07FF90E080A10181B19
:1034E0001D1A1A1A1A1A1A20261A207C4AE0FFF707
:1034F00049FF00281FD0207C3AE0FFF743FF002857
:1035000016D1207C002813D125E000F0C3FAF5E1A4
:103510002078F7E7FFF736FF1DE0207C00280AD06F
:10352000002905D007E0207C002804D1002902D022
:10353000012010E04DE000200DE0130001F04CF9F7
:10354000070C050E111B262E0C0000F0A3FA0099A3
:103550000198FDF799F92074D0E11AE100F09AFA88
:103560000CE0207C0028E6D000990198FDF78CF94A
:103570000028E0D0DCE7207C0028DCD0009901980E
:10358000FDF782F90028D6D1D2E758E1207C002847
:10359000CED100990198FDF777F9B3E7207C002898
:1035A000ECD0C5E7102804D0112804D0122AAED1DF
:1035B0000AE0227C03E0207C0028A8D001220099A8
:1035C000019800F09DFC99E1207C00289FD000220A
:1035D000F5E715383D79030001F0FEF8120A1215DF
:1035E000181B0F1E3C4C5B6A2D798185898D7D945B
:1035F00000F050FA13E0207484E000F04BFA1DE074
:1036000000F048FA29E000F045FA36E000F042FA0E
:1036100042E000F03FFA4EE0207C002870D02846BF
:103620000099FDF7B9F90546F9887879FDF7B4F9FD
:10363000854263D064E0207C002861D02846009950
:10364000FDF7AAF90546F9887879FDF7A5F98542CD
:1036500054D155E0207C002852D028460099FDF72F
:103660009BF90546F9887879FDF796F9854245DB9F
:1036700046E0B1E0207C002842D028460099FDF7C2
:103680008BF90546F9887879FDF786F9854235DCAE
:1036900036E0207C002833D028460099FDF77CF9DD
:1036A0000546F9887879FDF777F9854226DD27E028
:1036B000207C002824D028460099FDF76DF90546A6
:1036C000F9887879FDF768F9854217DA18E0207CE7
:1036D000002813D1A3E7207C00280FD1AEE7207C7F
:1036E00000280BD1B9E7207C002807D1C5E7207C52
:1036F000002803D1D0E7207C0028DCD001207AE725
:10370000002078E70225F9E03F791546C8280DD05A
:10371000DC2823D0DD282AD0FA28F3D12D48E9006F
:1037200008184030007EC0062AD508E02948E90084
:1037300008184030007EC00601D4002121E0207C22
:10374000002822D038460099FDF726F90146284680
:1037500000F07EFA284600F0F5F84CE71D48E90035
:1037600008184030007EC006E9D4012109E019485C
:10377000E90008184030007EC006E0D4022100E0D5
:1037800003212846FDF728FED9E7284600F07EFDF4
:10379000E0E73F790225342802D0372816D108E027
:1037A000207C002812D038460099FDF7F5F8401C1F
:1037B00007E0207C002809D038460099FDF7ECF896
:1037C000401E02463846009900F012FC96E00000C8
:1037D000E4140020CC0A00203D7979790291F9881F
:1037E0000191332814D035281BD038288AD1207C69
:1037F000002887D00298FDF7CFF8074628460099A1
:10380000FDF7CAF83A1A0199029800F0F1FB79E73E
:10381000207C0028FBD028460099FDF7BDF8024621
:10382000F1E7207C0028F2D028460099FDF7B4F893
:10383000054601990298FDF7AFF82A18E3E73A79AF
:1038400079790291F9880191797A03917D893628F5
:1038500006D0392812D03A281FD03B284DD131E06C
:10386000207C002849D010460099FDF795F80746BE
:1038700001990298FDF790F83A180CE0207C002896
:103880003BD010460099FDF787F80746019902984A
:10389000FDF782F83A1A29462CE0207C00282CD02B
:1038A00010460099FDF778F807B201990298FDF7E4
:1038B00073F800B247433A462946039800F098FB54
:1038C0003A1416E0207C002817D010460099FDF726
:1038D00063F807B201990298FDF75EF801B2384625
:1038E000FCF718FC02B20F462946039800F080FB53
:1038F0003A46691C039800F07BFB03253011410018
:103900000F48012308183107090F02898B40194617
:10391000114000D00121277C0830002F01D01A432C
:1039200000E09A43028076190698864200DA81E523
:1039300003494868401C4860002007B0F0BD000003
:10394000E4140020FEB50746402802DB0020C043F7
:10395000FEBD2C48F9000E1800964036348BE10667
:1039600001D40020FEBDA1063CD561063FD4264906
:10397000096800980A25406D0190081AA1070FD028
:10398000A107890F012905D0022905D0E143890744
:1039900005D005E0642503E07D25ED0000E01B4D2A
:1039A000A84224DB2946FCF7B5FB014615487A00FE
:1039B00012180B20800110188446808E019B40183D
:1039C00069435B18009980B24B650D21890151183C
:1039D000898E814203D8084640210C4334836146D6
:1039E000888604E0600602D5402084433483307E1C
:1039F000B9B24006C20F052000F082FA307E4006C0
:103A0000C00FFEBDCC0A00201001002010270000CE
:103A1000F7B50446FCF79BFF054602992068A942CA
:103A2000A16806DC4018029A0199FCF7BEFB0299D6
:103A300019E040182A460199FCF7B7FB29462046B1
:103A4000FCF7CCFC2046FCF782FF06460298471B99
:103A5000B7420DDCA16820683A464018019949191F
:103A6000FCF7A3FB39462046FCF7B8FC0298FEBDE4
:103A7000002E0CDDA16820683246401801994919D2
:103A8000FCF793FB31462046FCF7A8FCAD1928460D
:103A9000FEBD0000074A0F2011183F235B5C403138
:103AA000401E0B700028F7DC02494031087C08708A
:103AB00070470000CC0A002010B50C460A460146AB
:103AC0000348FFF7A5FF00F049FD204610BD0000A8
:103AD000CC02002010B50C460A4601460348FFF709
:103AE00097FF00F03BFD204610BD0000CC020020F7
:103AF00010B50C4600F09AFD204610BD04494968F7
:103B0000F0221140034A0909515CC8407047000087
:103B1000001002408557000803494968034A4905D7
:103B2000490F515CC840704700100240955700088B
:103B300010B5074841680C200140064805D004290B
:103B400004D0082901D100F009F810BD024810BDC9
:103B50000010024000127A00001BB70010B50C4C98
:103B60006168012212040B48114002D0914200D139
:103B70000948E16A0907090F491CFCF7B5FA6168B1
:103B80000F2292041140890C891C484310BD00008B
:103B90000010024000093D00001BB70070B5D417AB
:103BA000A40F0023A418A51003E09C000E59065191
:103BB0005B1C9D42F9DCD40F6B00A418651003E078
:103BC0005C000E5B06535B1C9D42F9DC104670BD29
:103BD0000920C006006901090F20884370470000D2
:103BE000F8B5002384468025DB4312480024214693
:103BF0002A464A43121817880F4EB74209D17E262B
:103C0000B75A0E4EB74204D15288A24201DD0B468C
:103C10001446491C0829EBDB082B06D26B43191804
:103C200080226046FFF7BAFF02E06046FEF7D0FD53
:103C30000020F8BD00C00008AA550000A55A0000E9
:103C40000B0702881B0F012199408A4302807047AD
:103C500030B5402802DB0020C04330BD0D4CC2000F
:103C600013191A464032157EAD0611D440000019D2
:103C70000D24A4010419A1860B240021A40100191C
:103C80008186054800685865108B20210843108301
:103C9000002030BDCC0A00201001002010B500F03B
:103CA00001F810BDF0B52E4FB868C007C00F4ED058
:103CB000F8682D4DC4B22B48C16E491CC166403016
:103CC000018D491C01852878002802D1204601F089
:103CD00063F828780026002819D12548234902785E
:103CE0008C540178491C01700D2C10D104460078C9
:103CF00001F052F820781F4908701F490120087010
:103D000026701E48067001201D490007486028786B
:103D100000281CD01B490878401C08701A48026F04
:103D2000521C02670878194A1278904210D3012079
:103D3000C0020921C90688612E701549012008704A
:103D40000E4908700A480670124980208862F0BD4A
:103D500011480978405C387301F01EF8F0BD00008E
:103D600000300140CC1100201C0000205402002033
:103D7000190000202D0000202C0000201800002039
:103D800000ED00E01B000020CC1000201A000020F5
:103D90002E000020001400483402002070B51A4C98
:103DA0006168491C616019490180A18841801849F6
:103DB0008A89828049698160112181831549C18383
:103DC000A1684A011449511800250B462A469E5CF9
:103DD000FF2E04D1521C202AF9D3002D10D020220E
:103DE000FCF7ECFBA0682060401CA06040010121B2
:103DF00089022030884201D90020A060002070BDD7
:103E0000202200F0AFFCEDE7AC000020AA55000036
:103E10004C100020A55A000000C8000870B50346E9
:103E20000E460807C10E1348002509180520C001D9
:103E30000818818A104C491C8182207A002817D1E9
:103E4000324619460D48FCF7B0F9A6710020E07122
:103E50000A48E179405C0A4908730121217200F0A7
:103E60009BFF08498020886100010921C9068862FA
:103E7000284670BDCC0A0020140000203402002027
:103E8000003001400014004810B514460A460128CD
:103E900002D0022806D00DE021461046FFF71AFE98
:103EA000054804E021461046FFF722FE0348816FD3
:103EB000491C8167204610BD7402002008030020C1
:103EC0000B0702881B0F012199400A4302807047AB
:103ED0000907090F01238B400188002A01D01943EB
:103EE00000E09943018070470907090F01238B40C7
:103EF0000188002A01D0194300E0994301807047EE
:103F000070B50B051B0E204C5B000D071C192D0F07
:103F1000030000F061FC09060B14191E22272C3146
:103F20003600FF292DD89520800003E0FF2928D8EE
:103F30009D20800020182946FFF7D6FF21E0FF29A9
:103F40001FD8A5208000F5E780291AD2FD20800027
:103F5000F0E7802915D20D48ECE7402911D2AD20B9
:103F60008000E7E740290CD2B5208000E2E78029F5
:103F700007D206482030DDE7802902D203484030CE
:103F8000D8E7002070BD0000CC0A00201404000017
:103F90000121C903034A002801D091627047916151
:103FA000704700000008004801218903034A0028E7
:103FB00001D091627047916170470000000800488D
:103FC0000121C903034A002801D091617047916221
:103FD000704700000008004801214903034A0028F7
:103FE00001D091627047916170470000000800485D
:103FF000F0B5304C4B001C1911239B01E61815231A
:104000009B01E51892B28A283DD00EDC294F4B0067
:10401000DF1909239B01FF188338030000F0DCFB44
:104020000714181C21262D46480099283ED006DC8E
:104030008B282CD08C2831D08D2839D133E0A12881
:1040400034D0FE2834D131E0102931DABA822FE0A1
:1040500010292DDABA862BE0102929DA0520C001B3
:1040600008E0082924DA0F20800114E008291FDA6B
:1040700001208002201882821AE0802918DAB28694
:1040800016E0AA8614E0802912DAB28210E04029F4
:104090000EDA0D2080012018828609E0402907DA17
:1040A0000B208001F7E7402902DAE8E78029E8DB06
:1040B0000020F0BDCC0A0020F0B58DB0002500F046
:1040C000E7FDFCF7D5FC059010213A4800F042FED0
:1040D0000790FCF7CDFC04901021364800F0E4FD79
:1040E0000690FCF7C5FC03901021324800F0FAFD61
:1040F0000190FCF7BDFC064610212E4800F00AFE98
:104100000090FCF7B5FC2C4A044690680121084356
:104110009060881E106129481061264B0021585C70
:104120001070491C1029FADB1768FCF7A1FC0B90F2
:104130000199009802970190214F0091781921A1CF
:10414000069B079A00F034FB45190B98A11B001B36
:1041500001910290039A04990398B21A431A0092AB
:1041600008460599421A781920A100F021FB44194C
:1041700008A8FEF723FA26484268012000040240FE
:104180003819134623A100F013FB0419381926A18E
:10419000089A00F00DFB01193846FFF78DFC01214C
:1041A0000D20FEF74DFB24490320886000200DB050
:1041B000F0BD0000895200080030024001A000005C
:1041C000140100200D0A435243202025303458208A
:1041D00020253034582020253034582020253034F4
:1041E000582020253034580D0A00000074696D6590
:1041F00020253034642020253034642020253034BC
:10420000642020253034642020253034640D0A00D9
:10421000001002404D61696E536F75726365202511
:1042200078202564200D0A00737973636C6B202558
:1042300064200D0A000000000000002030B50021BD
:10424000104D0846696042005219401C1181FF2838
:10425000F9DD002005220C4CD20143001B199B18EC
:10426000401C99821028F8DB0020112292014300A3
:104270001B199B18401C9986FF28F8DD0120286037
:10428000002030BDE4140020CC0A002010B54028E6
:1042900002DB0020C04310BD0B4BC100CA18114601
:1042A00040310C7EA4060DD54000C0180B2300241D
:1042B0009B01C0188486054800685065088B202241
:1042C00090430883002010BDCC0A0020100100207C
:1042D00010B5FCF7A1FCFCF785FE10BD70B594B0DD
:1042E00030216846FBF77AFF0024022501260E9450
:1042F000E8030990009605200F94C0040D940196E0
:104300000A900C9408950B956846FCF77DFE0028F2
:1043100003D0862115A000F049FA07200C900E94D6
:1043200001210D950F940CA8FCF73CFD002803D04B
:1043300092210EA000F03AFA109610A81296FCF7FF
:10434000BBFC002803D0A12108A000F02FFA4B20CD
:104350008001FDF703F80420FCF7FEFD0022114662
:10436000501EFCF7A5FC14B070BD00002E2E5C455D
:1043700078745F4650305C5372635C4253502E63D6
:1043800000000000134801680122114301604168E8
:10439000114A114041600168104A114001600168F2
:1043A000012292049143016041683F22120491432B
:1043B0004160C16A09090901C162016BFF2214321F
:1043C00091430163416B49084900416300218160C9
:1043D00070470000001002400CB8FF08FFFFF6FE17
:1043E00004480169C907C90F02D00121C94301610D
:1043F000704700000010004070B51B4CE0691B497D
:104400008006C00F11D01A4A01201060194A1060AE
:104410000869401C0861A28C4868401C4860174B22
:10442000154D18682A54401C1860E0690007C00F39
:1044300004D008202062C869401CC8612068C006FA
:10444000C00F07D0E069C006C00F03D01020206263
:1044500000F03CF8E0694006C00F03D04020206225
:1044600000F074F870BD00000038014074020020B4
:1044700060000020640000209C0300205800002001
:1044800010B5104CE069E0690007C00F05D00820A6
:1044900020620D48C169491CC1612068C006C00F77
:1044A00007D0E069C006C00F03D01020206200F0E2
:1044B0009DF8E0694006C00F03D04020206200F064
:1044C000E5F810BD00440040080300200548416A9B
:1044D000491C416204490968002901DD0121C167C5
:1044E000704700007402002058000020F8B5144DF9
:1044F0000C46064602212846FDF778FF1020009062
:10450000104B324602212846FDF75AFF224602216F
:104510002846FDF79DFF02212846FDF773FF0A4854
:1045200004630121417202212846FDF777FF054807
:10453000283881688022114381602046F8BD000040
:104540000000024028380140740200200248016A3D
:10455000491C0162704700007402002010B50A482F
:10456000407A00280DD1084C206F5834002808D11B
:104570002046FCF7D9F90146E26820688018FFF769
:10458000B5FF002010BD000074020020F8B5144DE6
:104590000C46064605212846FDF728FF002000901E
:1045A0003346104A05212846FDF70AFF2246052119
:1045B0002846FDF74DFF05212846FDF723FF0A4851
:1045C00044630121817205212846FDF727FF054834
:1045D000243881684022114381600020F8BD00002A
:1045E0000000024024440040080300200A480B4910
:1045F00000794058802180B2081A094901220860D8
:104600000849CA674A6A521C4A62002803DD012031
:1046100005490007486070479A52000804000240AC
:104620005C0000200803002000ED00E0F8B5144D08
:104630000C46064604212846FDF7D8FE10200090BF
:10464000104B324604212846FDF7BAFE22460421CB
:104650002846FDF7FDFE04212846FDF7D3FE0A4853
:1046600004630121417204212846FDF7D7FE054865
:10467000283881688022114381602046F8BD0000FF
:104680000000024028440040080300200248016A5C
:10469000491C0162704700000803002010B5054C5A
:1046A0000A46638821465B1C4380FBF787FF002096
:1046B00010BD0000007C000870B50C460B49411885
:1046C000002B08D00A4D4519012B03D0094B9B8ABA
:1046D000002B00D129460028204603D000F042F8E4
:1046E000002070BDFBF76AFFFAE7000000800008B9
:1046F00000A0000840120020F8B54188174A491C64
:104700004180154901807E2100250A52ED43802316
:1047100000221146124C002659430C19314603E081
:10472000675CFF2F04D1491C9942F9DB002E03D0AE
:10473000521C082AEDDB00E01546082D06D2084978
:104740005D436918802200F00DF803E080220449DF
:10475000FBF734FF0020F8BDAA550000A55A000061
:1047600000C00008F7B50D460646FCF73DFA029872
:104770000024870807E0A0003258411900230220D6
:10478000FCF7F4F9641CA742F5D802987C004708AE
:1047900007E06000325A411900230120FCF7E6F9D6
:1047A000641CA742F5D8FCF7D7F9FEBDFEE7000070
:1047B0000FB410B504A9074B02AA039800F028F81B
:1047C000044602A9002000F05DFA204610BC08BC97
:1047D00004B01847854C000830B47446641E257830
:1047E000641CAB4200D21D46635D5B00E31830BC25
:1047F000184702E008C8121F08C1002AFAD1704702
:104800007047002001E001C1121F002AFBD1704750
:10481000FFB591B00F460546002606E025280AD0D0
:10482000149A139990476D1C761C28780028F5D1AE
:10483000304615B0F0BD002400940121F34A0294E3
:1048400000E004436D1C2B780846203B9840104242
:10485000F7D128782A280ED0022128780246303A4B
:10486000092A15D8009A0A235A43303A80180C4373
:104870006D1C0090F1E701CF0090002805DA0120BF
:1048800040030443009840420090022004436D1C02
:1048900028782E2815D10420044368786D1C2A2816
:1048A0000AD101CF6D1C02900BE002990A225143FC
:1048B000303940186D1C029028780146303909299A
:1048C000F3D928786C2810D006DC4C281AD0682838
:1048D0000ED06A2817D104E0742813D07A2812D198
:1048E00010E00120400504430CE00121090501E02E
:1048F000032109050C436978814203D10120000599
:1049000024186D1C6D1C287803906E281ED00CDCBA
:10491000632831D004DC00288AD0582811D1B2E0B5
:1049200064287BD069280CD178E073282DD004DC72
:104930006F2870D0702804D1A7E075286CD0782833
:104940006BD0149A13999047761C62E06002400F76
:10495000022807D003280AD0042838680AD0066045
:104960003F1D56E03868F11706604160F8E7386887
:104970000680F5E70670F3E738786946087400208A
:10498000487404A80390012003E0386803900020D5
:10499000C0433F1D61070FD5002101E00199491C6B
:1049A000029A0191914213DA8142F7DB019A03994D
:1049B000895C0029F2D10BE0002101E00199491C3A
:1049C00001918142FADB019A0399895C0029F5D1B2
:1049D00001990098139A401A00902146149B00F008
:1049E0003BF901998019461807E00398039900786C
:1049F000491C0391149A139990470198401E019005
:104A0000401CF2D12146149B139A009800F014F92F
:104A100086196D1C09E741E033E034E00A200021EB
:104A2000049005916002410F022905D001CFC21701
:104A30009446032905D007E0FF1DFF08FF0003CFC0
:104A400006E000B2C2179446042902D140B2C11751
:104A50008C4600226146944506DA0A46002140420F
:104A600091418C462D2102E0210504D52B216A4677
:104A70001176012103E0E10701D02021F7E7019140
:104A800054E00A200BE0102009E0102004900021DF
:104A90000420044308200591029003E0082000212F
:104AA000059104906002410F022905D001CF002238
:104AB0009446032906D006E0FF1DFF08FF0003CF40
:104AC0008C4603E080B2042900D1C0B200210191DC
:104AD00021072BD50399702906D0049A1021059B34
:104AE0004A401A4305D00EE040216A461176012162
:104AF00008E06146014306D030216A4611760399E9
:104B0000517602210191049A0821059B4A401A43DB
:104B10000CD16146014301D1610707D530216A46B6
:104B20001176012101910299491E02910399582998
:104B300004D037A103910FA90F910DE039A1F9E736
:104B40006146059B049AFBF75EFB039B8C469B5CCE
:104B50000F9A521E0F92137061460143F0D10F98C5
:104B600007A9081A20300390600704D5012000042B
:104B70008443029801E0012002900399884201DDFC
:104B8000401A00E00020411802900198091800988E
:104B9000401A0090E00306D42146149B139A009813
:104BA00000F05AF886190020049008E006A9085C75
:104BB000149A139990470498401C761C049001990C
:104BC0008842F3DBE0030CD52146149B139A00982E
:104BD00000F042F8861904E0149A302013999047A7
:104BE000761C0299481E02900029F5DC08E00F9817
:104BF0000F990078491C0F91149A13999047761CCD
:104C00000399481E03900029F1DCFBE60928010006
:104C10003031323334353637383961626364656632
:104C200000000000303132333435363738394142F4
:104C30004344454600000000F8B5044600251E46E2
:104C40001746880404D405E039462020B0476D1C7F
:104C5000641EF9D52846F8BDFFB50446002581B08D
:104C60001E46C80301D5302700E02027880404D55C
:104C700005E038460399B0476D1C641EF9D52846F7
:104C800005B0F0BD0A68531C0B601070704700003F
:104C900010B50A2101A0FEF70FFF10BD1B5B324AC1
:104CA0001B5B303B3048000030B503460B48002901
:104CB00000D101210A4C491E0ED31A78504000221F
:104CC000C50702D04008604000E04008521CD2B244
:104CD000082AF5D35B1CEEE730BD0000FFFF0000A3
:104CE00001A0000070B50A4DFF23EE1D1A46F936EB
:104CF00005E0047854402A5D5A40335D401C0C4660
:104D0000491E89B2002CF4D11802104370BD000076
:104D1000A054000870B504460C4800220C4E11E067
:104D20002378521C1D4645402D07ED0E755B00098A
:104D30004540180968400007C00E305A2B095840FA
:104D400092B2641C8A42EBD370BD0000FFFF0000EA
:104D50006057000810B5084A084B07E00478544033
:104D60002406E40D1C5B120A6240401C491EF5D269
:104D7000D04380B210BD0000FFFF0000A052000829
:104D800006C00021016041608160C16001220261B2
:104D90004161084670470000074910B54A8D0B462F
:104DA0004C3BD054488D401C80B24885642801D3C8
:104DB0005120488510BD00000C120020FE4F8AB023
:104DC0000126FF203E830530FC4B80220090991A7B
:104DD000FB48FCF721FB4020FA4B0246191A0090D1
:104DE000F948FCF719FBFBF71FFF0021F74A0D46B6
:104DF0006020484380184560856005614561856194
:104E0000C561056285624562C562491C0563092961
:104E1000EEDBEF4CEF482563C06A6062EE48006845
:104E2000A062EE48406AE062FFF758FAED49EC48AC
:104E30000860FCF701FBFDF729FDFDF713FDFDF709
:104E400065FAE948FEF7CCFEDB480683FEF7C0FEB4
:104E5000214680390791102108430799E34A4867A2
:104E60000107090FC006E248117003D50670E1483A
:104E7000057002E00570DF480670DF4F3970FBF700
:104E800047FCDA48E12100783870DC4801270770D8
:104E9000DB4889020160FDF73DFEFDF7CDFEFDF721
:104EA000A9FDD8484168402631434160FDF788FD9F
:104EB000FDF706FED448016839430160D348016814
:104EC0002022114301600168102739430160016805
:104ED000314301608021CE48FFF758FBCD4801687F
:104EE000394301600168314301600A20FBF7D6FDB8
:104EF0000120FFF771F80020FFF756F80020FFF7B8
:104F00005FF8FFF7D9F8FBF7B3FDAB4E606235826F
:104F1000308A012803D1FCF739FAFFF78FF95A21BB
:104F2000BD48089041840126BC4D00272F706E704B
:104F3000FBF79EFD2861FBF769FE07990690C8679D
:104F4000FBF70AFCFBF794FD68612078C006C00EF1
:104F5000022818D1FBF7AAF9B14801680029B14924
:104F60000A680AD0002A0ED100680860AE480068BE
:104F7000AE490860FEF716FA05E0002A03D0006883
:104F80000860FEF727FA8C48008A01280FD198485C
:104F9000007800280BD08848818A00291FD0A449B6
:104FA000A960C18AA3480160A868FEF71BFA606A7D
:104FB00069696162081AA062E16A884200D2E0620F
:104FC000216B884200D92063FBF752FDA861884815
:104FD0000078002818D0984900200B780BE09749FA
:104FE000DEE7974913220918520189180A7D95496D
:104FF00009184A70401C9842F3DB7F48007800286B
:1050000002D00220FCF710FB0698800401D52E7018
:1050100000E02F700698000501D56E7000E06F70FB
:1050200074480078002818D00220FCF7C5FC60689E
:10503000002801D184480770834801780898818648
:1050400082480168890401D52E7000E02F70006845
:10505000000501D56E7000E06F706068002801D017
:10506000401E6060A068002801D0401EA060524829
:10507000008B00283FD06878FEF7AEFF6878FEF717
:1050800093FF6878FEF784FF6878002801D101203B
:1050900000E00020FEF794FFFBF7EAFCE861FBF775
:1050A000E7FC2862FBF7E4FC0A2168620846FBF78C
:1050B0000BF80020401C4028FCDB20686449401CA1
:1050C0002060086800282FDD3D4AD26F002A2BD0CF
:1050D00082B260490120FDF777FE002805D05C48C8
:1050E0005C4902680120FCF77DFD5948076034489F
:1050F000C7676F602CE0606800280CD06878FEF706
:105100006BFFA068002808D06878FEF74DFF68782C
:10511000FEF73EFFBDE72878F1E70020FEF744FFE9
:105120000020FEF735FFB2E74B49686888420DD989
:10513000364841680122120511434160416852001E
:1051400003235B0599431143416001E0401C686003
:1051500028480078002802D00020FBF79FFC182286
:105160003E496846FBF721F83D4F00206D461E4939
:105170004200511840310A891105130B1207090E1C
:10518000120F00296ED0002B02D0012B06D069E04F
:105190002B4B591809239B01C91804E0284B5B18B5
:1051A000132149015918C97C33469340194259D0FB
:1051B00081006958B96158E040120020E0120020D7
:1051C000740200202414002008030020BC050020E5
:1051D0004C10002080F7FF1F4C0000200010024000
:1051E00010270000300000204C0A00206C00002036
:1051F0006800002069000020730000206D0000207E
:1052000050000020003001400010004000380140F4
:105210001C040020004400400C0D0020DC00002095
:10522000D0000020D400002034000020D80000204E
:1052300000A00008080100201700002000800008DE
:10524000CC0A0020AC0400209C0400208400002034
:10525000580000209C030020C02709004857000880
:105260000004004881006958B962401C062800DA31
:105270007DE703490148086056E60000AAAA00003D
:1052800000300040081C30445811223344556677E2
:105290008899AABBCCDDEEFF0000081C3044580002
:1052A0000000891112239B322446AD573665BF7426
:1052B000488CC19D5AAFD3BE6CCAE5DB7EE9F7F8D6
:1052C0008110080193331A22A5562C47B7753E6406
:1052D000C99C408DDBBF52AEEDDA64CBFFF976E8B6
:1052E00002218B30100299132667AF763444BD55E6
:1052F0004AADC3BC588ED19F6EEBE7FA7CC8F5D996
:1053000083310A2091121803A7772E66B5543C45C5
:10531000CBBD42ACD99E508FEFFB66EAFDD874C975
:1053200004428D5316619F702004A9153227BB36A5
:105330004CCEC5DF5EEDD7FC6888E1997AABF3BA55
:1053400085520C4397711E60A1142805B3373A2685
:10535000CDDE44CFDFFD56ECE9986089FBBB72AA35
:1053600006638F7214409D512225AB343006B91765
:105370004EEFC7FE5CCCD5DD6AA9E3B8788AF19B15
:1053800087730E6295501C41A3352A24B116380745
:10539000CFFF46EEDDDC54CDEBB962A8F99A708BF5
:1053A000088481951AA793B62CC2A5D33EE1B7F025
:1053B0004008C919522BDB3A644EED5F766DFF7CD5
:1053C000899400859BB712A6ADD224C3BFF136E005
:1053D000C1184809D33B5A2AE55E6C4FF77D7E6CB5
:1053E0000AA583B4188691972EE3A7F23CC0B5D1E5
:1053F0004229CB38500AD91B666FEF7E744CFD5D95
:105400008BB502A499961087AFF326E2BDD034C1C4
:10541000C3394A28D11A580BE77F6E6EF55C7C4D74
:105420000CC685D71EE597F42880A1913AA3B3B2A4
:10543000444ACD5B5669DF78600CE91D722FFB3E54
:105440008DD604C79FF516E4A9902081BBB332A284
:10545000C55A4C4BD7795E68E11C680DF33F7A2E34
:105460000EE787F61CC495D52AA1A3B03882B19364
:10547000466BCF7A5448DD59622DEB3C700EF91F14
:105480008FF706E69DD414C5ABB122A0B992308344
:10549000C77B4E6AD5585C49E33D6A2CF11E780FF4
:1054A00000C1814001C0804101C0804100C18140F4
:1054B00001C0804100C1814000C1814001C08041E4
:1054C00001C0804100C1814000C1814001C08041D4
:1054D00000C1814001C0804101C0804100C18140C4
:1054E00001C0804100C1814000C1814001C08041B4
:1054F00000C1814001C0804101C0804100C18140A4
:1055000000C1814001C0804101C0804100C1814093
:1055100001C0804100C1814000C1814001C0804183
:1055200001C0804100C1814000C1814001C0804173
:1055300000C1814001C0804101C0804100C1814063
:1055400000C1814001C0804101C0804100C1814053
:1055500001C0804100C1814000C1814001C0804143
:1055600000C1814001C0804101C0804100C1814033
:1055700001C0804100C1814000C1814001C0804123
:1055800001C0804100C1814000C1814001C0804113
:1055900000C1814001C0804101C0804100C1814003
:1055A00000C0C101C30302C2C60607C705C5C404C3
:1055B000CC0C0DCD0FCFCE0E0ACACB0BC90908C833
:1055C000D81819D91BDBDA1A1EDEDF1FDD1D1CDC23
:1055D00014D4D515D71716D6D21213D311D1D01093
:1055E000F03031F133F3F23236F6F737F53534F483
:1055F0003CFCFD3DFF3F3EFEFA3A3BFB39F9F838F3
:1056000028E8E929EB2B2AEAEE2E2FEF2DEDEC2CE2
:10561000E42425E527E7E62622E2E323E12120E052
:10562000A06061A163A3A26266A6A767A56564A442
:105630006CACAD6DAF6F6EAEAA6A6BAB69A9A868B2
:1056400078B8B979BB7B7ABABE7E7FBF7DBDBC7CA2
:10565000B47475B577B7B67672B2B373B17170B012
:105660005090915193535292965657975595945402
:105670009C5C5D9D5F9F9E5E5A9A9B5B9959589872
:10568000884849894B8B8A4A4E8E8F4F8D4D4C8C62
:1056900044848545874746868242438341818040D2
:1056A000030E0201000100010401000600000000D9
:1056B0000000000000000600AA55000000010000E4
:1056C00000000000010001000009000000000000CF
:1056D00000000200000000090000000000000000BF
:1056E00000000000000000000000000000000000BA
:1056F00010101010101010101010101010101010AA
:105700001000200030004000500060000300000046
:105710000400000005000000060000000700000073
:1057200008000000090000000A0000000B00000053
:105730000C0000001100A55AAA550000000000004E
:10574000000000000000000000040000000800004D
:105750000010000000200000004000000080000059
:10576000000001CC01D8001401F0003C002801E445
:1057700001A0006C007801B40050019C0188004435
:10578000081C304458000000000000000001020323
:1057900004060708090000000001020304000000DD
:1057A000C05700080000002014010000F247000864
:1057B000D458000814010020FC1900000248000819
:1057C00000000000000000000000000000000000D9
:1057D00001000000000008080000000000000000B8
:1057E00000000000000000000000000000000000B9
:1057F0001027000000000000000000000000000072
:105800000000000000000000000000000000000098
:105810000084030040420F00000000000000000070
:105820000000000000000000000001000000000176
:105830000101000000000000000000000000000066
:105840000000000000000000000000000000000058
:105850000000000000000000000000000000000048
:10586000010000000000000000000000FFFFFFFF3B
:105870000000000000000000000000000000000028
:105880000000000000000000000000000000000018
:105890000000000000000000000000000000000008
:1058A0000000000000800008000000000000000070
:1058B00000000000000000000000000000000000E8
:1058C000000000000100000097000000001BB7006E
:0458D00000000000D4
:04000005080000B53A
:00000001FF
